:020000040000FA
:0200000048288E
:080008000900831203134830C4
:100010008600AA308700630005282E307007840010
:10002000000820182829002A2E30700784000008B4
:1000300028290310290D2907A1000310210DA10073
:10004000210D08006400FF3087001C2186003A3033
:10005000840000088700F8308407800803193D28D1
:1000600005183B2800000000000000000000000010
:10007000800B32283D28800B3B28393004020319BD
:100080004428093084072928FF30870086010800AA
:10009000FF3087008601850110108B018312031742
:1000A0009E019F0195018316031374128E1C741612
:1000B000013085008601870161308F008C01831239
:1000C00003138C012830900010147716FF30A50020
:1000D000741E6E28F4010C30A9008028741C772847
:1000E00074102908C200F4150B30A90080284208BA
:1000F000F419A900F411A90A29080A3C031CA90152
:10010000831603138E14831203130E300F07AD00F2
:100110001920A8000023F5002808A300F4142308E0
:10012000A8000023F2000023A2000023F300002314
:10013000AE000023AF000023B0000023B100002375
:10014000A0000023C3000023C7000F39C600470EDC
:100150000F39C7000023A800F41CB0282E0828215E
:100160007208F100A7014608C4004708C5002D0821
:100170000F02031DB7280E300F07AD00F001201E3F
:10018000D7281420BA000D20BB00FF30BC00BD00F2
:10019000BE00BF00C000C1002708B300C83CB200C9
:1001A000B401B501B601B701B801B901DA282F08C9
:1001B000282123252220F00A701DBF28A50303193A
:1001C00074144308A707C40BE828A70A4608C4000C
:1001D000C50BED28A70A4708C500F10BB728201E5C
:1001E0000129F0012E308400800A000873020318F0
:1001F000FC28220880007415840AF00A701DF42877
:1002000003292E080022741DB0287411201D122904
:10021000831603138E10831203138601FF308700A9
:1002200063004828A0197F28F50B1929A90803198C
:100230008A28A01CB0288F287008F60001308A0098
:100240007608820780344034203410348A1105281F
:10025000F60001308A0076088207FF340034FF344C
:10026000FF3477347734FF34BB34BB34FF34DD34B0
:10027000DD34FF34EE34EE3477347734BB34BB34C2
:10028000DD34DD34EE34EE347F347F340F3400342B
:100290000F347F347F340F3400340F34FF34FF3495
:1002A000F034FF340F34FF34FF340F34FF34F034B4
:1002B00000340034FF34FF34FF34FF34FF34FF34A4
:1002C000FF34FF34FF34FF34FF34FF34FF34003495
:1002D0000034FF34FF34FF34882CB32CFE34FC345C
:1002E000F934F334E734CF349F343F347F347F34F0
:1002F0003F341F34AF345734AB345534AA34003450
:10030000FF34FF34FF34FF34FF34FF34FF34FF3455
:10031000FF34FF34FF34FF34FF347734BB345534BB
:10032000AA340034FF34FF34FF34FF34FF34FF3489
:10033000FF34FF34FF347F34BF345F34AF3457347D
:10034000AB345534AA340034FF347F347F34FF3467
:10035000FF34FF34FF34EE34EE34FF34FF34FF3427
:10036000B634DB34DB346D346D34B6346D34DB34A9
:10037000DB34B634B6346D34003400348034833426
:10038000C734EF34EF34003400341134333477346D
:10039000FF34FF340034003401348334C734EF3485
:1003A000FF34FF34F734FF34EF34DB34BD34FE3434
:1003B0007F34FF34FF34FF347734FF34BB34DD3413
:1003C000FF34FF34FF34FF34FF34C734BB347D3493
:1003D000FE34FF34FF34FF34FF34C734BB347D3484
:0A03E000FE34C32DC92D8A11052833
:10040000F60002308A00760882070034FF34FF3499
:1004100077347734FF34BB34BB34FF34DD34DD3420
:10042000FF34EE34EE34FF347734BB34BB34DD3488
:10043000DD34EE34EE3477347F340F3400340F344F
:100440007F347F340F3400340F347F34FF34F03482
:10045000FF340F34FF34FF340F34FF34F034FF34F3
:100460000034FF34FF34FF34FF34FF34FF34FF34F3
:10047000FF340034FF34FF34FF34FF3400340034E1
:10048000FF34FF34FF34FF34E02C0800FC34F9342F
:10049000F334E734CF349F343F347F347F343F34F8
:1004A0001F34AF345734AB345534AA340034FF34DE
:1004B000FF34FF34FF34FF34FF34FF34FF34FF34A4
:1004C000FF34FF34FF34FF347734BB345534AA345F
:1004D0000034FF34FF34FF34FF34FF34FF34FF3483
:1004E000FF34FF347F34BF345F34AF345734AB3420
:1004F0005534AA340034FF347F347F34FF34FF3462
:10050000FF34FF34EE34EE34FF34FF34FF34FF3475
:10051000DB34DB346D346D34B634B634DB34DB3489
:10052000B634B6346D346D34003480348334C7341B
:10053000EF34EF34FF340034113433347734FF3484
:10054000FF34FF34003401348334C734EF34FF34D4
:10055000FF34F734F734EF34CB349934BC347E3481
:100560007F34FF34FF3477347734BB349934CC3460
:10057000FF34FF34FF34FF34C734833439347C34E0
:10058000FE34FF34FF34FF34C734833439347C34D1
:0A059000FE34E22D08008A11052850
:100600002808A80A032BF60003308A007608820720
:100610002C34083477348E34893483347D34773401
:100620001234193400340C34D13401343F344134A1
:100630003F34403487340A340034003400341834F2
:100640000B3418340F3416340F340F340F340F3486
:1006500010340834033424340634143441347634EA
:10066000653465345334413412340A340034303440
:100670000A34233403340E34033403340934093484
:100680001034053452343C340C341E34A434C33496
:10069000BC34B434AC34A434123406346234483438
:1006A000D13401343F3441343F34403487340A3448
:1006B00001340034003454340C34123417343E34D2
:1006C00035342B342134173412340B34093460346C
:1006D000D13401343F3441343F34403498340A3407
:1006E0000134003400346C3403340134C434C6346F
:1006F000C434C53400340034003400340034783459
:1007000005348C34003402340034003400340034B6
:1007100010340134A3340034013408348F34A3344A
:100720009D349D3496348F3416341934003490340B
:1007300001346434003400340034003400340034B4
:0C0740001A340234003400348A110528F9
:10080000F60004308A00760882070034013404348C
:10081000063409340B340E341034123415341734C2
:100820001A341C341F3421342434263428342B3415
:100830002D34303432343434373439343B343E346C
:10084000403442344534473449344C344E345034C7
:1008500052345534573459345B345E346034623426
:100860006434663468346A346C346E34713473348E
:100870007534773479347A347C347E3480348234FD
:1008800084348634883489348B348D348F34903476
:10089000923494349534973499349A349C349D34FA
:1008A0009F34A034A234A334A534A634A734A93489
:1008B000AA34AB34AD34AE34AF34B034B134B23426
:1008C000B434B534B634B734B834B934BA34BA34CD
:1008D000BB34BC34BD34BE34BF34BF34C034C13487
:1008E000C134C234C334C334C434C434C534C5344D
:1008F000C534C634C634C634C734C734C734C73425
:10090000C834C834C834C834C8348A110528000033
:10091000300883160313E2000130E3006208630528
:10092000031D952C0310E30D8E2C6208E3070310C2
:10093000E30DA03084002030E000FB248000840A16
:10094000FB24620580000310000D003A03196308C0
:100950008000800C840AE00B9D2C831203138A1103
:100960003108A6000800200883160313E3000310D3
:10097000700DE100E10DE10D610DAF3E8400083026
:10098000E0000301801BD02C84030008631CCC2CE6
:100990000301801BC830CF2C801B00090024840A6F
:1009A000E10084030403F6006008803C84006108D1
:1009B000800076088400E00BC12C8312031308002A
:1009C000831603132030E000DF30840000087F39F5
:1009D00084038007031CF02C840A80308006840383
:1009E0008403E00BE62C83120313A60B08003108E6
:1009F000A60074150800770D770D771A013AF71ADB
:100A0000013AF719013AF700080033308400040A6C
:100A1000AA000008840300020318152D2A08840088
:100A2000393C031C0800AA0A092D03190E2D0002E7
:100A3000000680060006840A800084033230040227
:100A40000319840A092D783084000830AA000008B0
:100A5000A100C2308407FF308000F83084072108ED
:100A6000800047308407AA0B272D05258030AA0077
:100A70007830840000080319522DAB000408AC0044
:100A80003230840000082B02031C502D08308407EC
:100A90002A088006F93084073A300402031D422DEB
:100AA0002C088400840A0310AA0C031C3A2D07307A
:100AB000AA00383084000008840A8002840384037A
:100AC000AA0B5B2D08003108A6003008831603131B
:100AD000B800A03084000830B900FB248000840AEC
:100AE000FB243805013E8000840AFB240739063EBA
:100AF0008000840AE00B6D2D831203138A11080015
:100B0000200883160313E3000310700DE100610D4C
:100B1000E107A53E84000230B9000301801B982D37
:100B200084030008801B00090024840A6318C8306D
:100B3000E10084030403F6006008803C840061083F
:100B4000800076088400E00BC12C83120313080098
:100B5000831603132030E000DF30840000087F3963
:100B600084038007031CB82D840A80308006840328
:100B70008403E00BAE2D83120313A60B080031088B
:100B8000A60074150800831603130130C100C000CD
:100B9000E22D831603130830C4000310700DC20049
:100BA000C20D420DA73EC20084000008C3004408E5
:100BB000773E8400430880004203C40BD32D831288
:100BC0000313080083160313C00B002E2830C00047
:100BD000C10B002E74151E30C1000730C400C83090
:100BE00084002D308000840A043EC40BF22D203096
:100BF000C400A03084008001840AC40BFB2D292E80
:100C0000410B292EA001A801B8011D30C5000430F8
:100C1000C600C830C7001E3040024008031CC50093
:100C2000142ECE30C707C603C61B112EC2011D30BD
:100C3000C4004208C20A732647088000C503C51FC6
:100C4000262EC603C61B262ECE30C707C40B192E70
:100C5000702E26304002031C302E023CB800352E88
:100C6000213E0630031CCE30B8070730C400CE301A
:100C70008400C201800B3F2E283080004A2E0930AC
:100C8000000203184A2E3230C20005300002CE3076
:100C9000031CC2000403C3004408B83E8400420899
:100CA000800743088400C40B392E41081D3C031CF7
:100CB000702EC50006304E020318632E45087326B9
:100CC0003F08C83C80004E03E43E0318C50A4508AF
:100CD0000319702E45037326C8308000C50B6A2E99
:100CE000831203130800762684000800F6000630FD
:100CF0008A0076088207A734AF34B334B734A634F9
:100D0000AE34BF34B234B634A534AD34BE34B134AD
:100D1000B534BD34A434AC34B034B434BC34A334AE
:100D2000AB34BB34A234AA34BA34A134A934B934B4
:0A0D3000A034A834B8348A11052855
:00000001FF
